:020000040000FA
:1000000025003B0A3000460500000000000000000B
:1000100000000000000000000000000000000000E0
:100020004604000000000000000000000000000086
:100030000000F002030A0008300011023200000044
:1000400000000000000000000000000000000000B0
:1000500000000000000000000000000000000000A0
:1000600000000000000000000000F2021F0A320041
:10007000F0021F0A000804006600000C06000200DF
:10008000020C3300D302480A0F0C3100A70C1C09E4
:100090005A0C02090F0C3100490C1C091A0C0209F8
:1000A000120C3100030C1C09150C0209020C310062
:1000B0003F0C1C091A0C0209F302420A140C31000D
:0600C000A70C1C09400A18
:021FFE00EA0FE8
:00000001FF
